:100000000C944A010C9482010C9482010C9482019C
:100010000C9482010C9482010C9482010C94820154
:100020000C9482010C9482010C944B1D0C941D1EA7
:100030000C942A180C9482010C9482010C94820175
:100040000C9482010C9482010C9482010C94820124
:100050000C9482010C94B2180C9482010C948201CD
:100060000C9482010C9482010C9482010C94820104
:100070000C9482010C9482010C9482010C948201F4
:100080000C9482010C9482010C9482010C948201E4
:100090000C9482010C9482010C9482010C948201D4
:1000A0000C9482010C9482010C948201680468040F
:1000B00094049404FC041A05320632062505BE0594
:1000C000CF05CF058A1EB11EA91FB11EA91FFD1E97
:1000D000201FA91F771F861F5F0060006100570067
:1000E0005C005D005E00560059005A005B00550040
:1000F00001516200630028005300A75D0100540015
:10010000005CA85D010001000100A95D0100010083
:100110000100AA5D010001001203430072006100AA
:1001200077006C0050006100640000001E0357005F
:100130006F006F0064004B006500790073002E00B3
:1001400063006C00690063006B0000000403090495
:1001500009023B00020100A0FA09040000010301AA
:100160000100092111010001224000070581030857
:100170000001090401000103000000092111010030
:100180000122B600070582032000011201000200CF
:10019000000008EDFE706001000102000105010988
:1001A00002A10185020901A100050919012908150B
:1001B00000250195087501810205010930093115F5
:1001C00081257F95027508810609381581257F955F
:1001D0000175088106050C0A38021581257F9501F5
:1001E00075088106C0C005010980A10185031901B8
:1001F0002AB700150126B700950175108100C005CA
:100200000C0901A101850419012AA002150126A0EB
:1002100002950175108100C005010906A10185063E
:10022000050719E029E715002501950875018102E8
:100230000507190029EF1500250195F075018102C8
:1002400005081901290595057501910295017503A8
:100250009101C005010906A101050719E029E7156B
:100260000025019508750181029501750881010538
:1002700007190029FF150026FF0095067508810063
:100280000508190129059505750191029501750368
:100290009101C00011241FBECFEFDAE0DEBFCDBF59
:1002A00004B603FE18C080917F0290918002A09155
:1002B0008102B09182028730904BA740B04B59F435
:1002C00010927F021092800210928102109282029C
:1002D000E0E0F8E3099511E0A0E0B1E0E8EBF0E43C
:1002E00002C005900D92A438B107D9F722E0A4E826
:1002F000B1E001C01D92AF37B207E1F70E94F411DF
:100300000C945A200C940000FB01883A2DE59207CA
:10031000A1F020F4873A9D4549F025C0893A2DE5A2
:10032000920799F08A3A9D45B9F01DC082818823D1
:1003300011F02C9A06C02C9808958281882319F018
:100340002D9A80E008952D9808958281882311F0D8
:100350002E9AF7CF2E9808958281882311F02F9A34
:10036000F0CF2F98089581E0089584B1806F84B90B
:1003700085B18F7085B9089581E008950C9484014A
:1003800008950C94C0011F93CF93DF9300D000D049
:100390001F92CDB7DEB749835A836B8330918701B3
:1003A00089819A81311114C0662359F0222349F0C2
:1003B0000E946D08182F682F89819A810E94180861
:1003C00003C00E944208182F69817A81812F04C0DE
:1003D0000E946D0869817A810F900F900F900F90A5
:1003E0000F90DF91CF911F910C94880FFC01262F65
:1003F000408151816281738184810C94C30181E0C9
:100400000895CF93DF93EC0160E00E94F601BE01F6
:10041000DF91CF910C94C1010C94B3100C94B110E6
:1004200008950E94C2060E9410022FEF84E39CE010
:10043000215080409040E1F700C000000C94D81893
:100440000F931F93CF93DF938C0161E00E94F6011D
:10045000EC01B8010E94BE018823F1F1B801CE0180
:100460000E9476168823C1F1B801CE010E948A1439
:10047000882391F1B801CE010E94D215882361F141
:10048000F8018281882309F1CB358DE5D807C1F0C9
:1004900050F4C115FCE5DF0781F0CF3DDC45A9F440
:1004A0000E949E0D19C0CC35EDE5DE0761F0CD351B
:1004B000DD4559F40E94E70C08C00E9411020CC0EF
:1004C0000E94F00C02C00E94F30CC801DF91CF9192
:1004D0001F910F910C94BC0180E0DF91CF911F918F
:1004E0000F9108950E940D180C948B020E948E02A9
:1004F0000C94131808950C947A0281E008950C94DA
:100500007D020895CF93C82F0E947B028C2F0E94FA
:100510007F02CF91089580E00C9482020E94D2164F
:100520000C9482020E94D21690918601891721F0C4
:10053000809386010C9482020895CF93DF93CDB708
:10054000DEB72B970FB6F894DEBF0FBECDBF4F833B
:10055000588769877A878B8761110E94330C9E01C7
:100560002F5F3F4F86E0F90111928A95E9F785E008
:10057000FE013796D90101900D928A95E1F78981A4
:100580009A814C815D81452B31F09F3F31F491E0A0
:100590008F3F19F403C091E001C090E090FF09C0C3
:1005A00049815A816B817C818D819E810E94540B8F
:1005B00005C0C9010E94FF018111F2CF2B960FB631
:1005C000F894DEBF0FBECDBFDF91CF910895FC013F
:1005D000808191810E94AF080895CF93882309F408
:1005E000A4C0C82F8238C1F40E94D21681FD9DC0DC
:1005F00069E380910201909103010E94C8170E9453
:10060000550C2FEF81EE94E0215080409040E1F7AF
:1006100000C0000069E319C0833801F50E94D216BA
:1006200080FD83C063E580910201909103010E94E7
:10063000C8170E94550C2FEF81EE94E021508040A6
:100640009040E1F700C0000063E5809102019091C5
:1006500003010E94D317CF910C94550C8438C1F438
:100660000E94D21682FD61C067E4809102019091E0
:1006700003010E94C8170E94550C2FEF81EE94E0F1
:10068000215080409040E1F700C0000067E4DDCFDA
:100690008CEF8C0F813AD0F46C2F809102019091F5
:1006A00003010E944817882349F06C2F80910201B2
:1006B000909103010E94D3170E94550C6C2F8091DA
:1006C0000201909103010E94C817C5CF80E28C0FF0
:1006D000883048F4C77081E001C0880FCA95EAF7F6
:1006E0000E94160CB8CFEBE5EC0FE33040F4F0E0DD
:1006F000E95BFE4F808190E0CF910C940617E8E50E
:10070000EC0FE73150F4F0E0EE0FFF1FE75EFE4F15
:1007100080819181CF910C941C17CD3E30F08C2FAD
:100720000E947912CF910C944B13CF910895882396
:1007300009F464C0823879F40E94D21681FF5EC049
:1007400069E380910201909103010E94C8170E9401
:10075000550C69E310C08338B1F40E94D21680FFB3
:100760004DC063E580910201909103010E94C8177A
:100770000E94550C63E580910201909103010E9453
:10078000D3170C94550C843879F40E94D21682FF4A
:1007900035C067E480910201909103010E94C8175F
:1007A0000E94550C67E4E7CF9CEF980F913A10F444
:1007B000682FE1CF90E2980F983050F4877091E065
:1007C00001C0990F8A95EAF7892F0E941C0CD9CF96
:1007D0009BE5980F933020F480E090E00C9406178E
:1007E00098E5980F973120F480E090E00C941C1766
:1007F0008D3E20F00E94D4120C944B1308951F9349
:10080000CF93DF93182FEB010E94ED02209741F068
:100810008FE99FE00197F1F700C000002197F6CF24
:10082000812FDF91CF911F910C949703893319F099
:1008300060E070E002C060E570E00C94FF03882384
:1008400021F00E94160C0C94550C0895882321F079
:100850000E941C0C0C94550C0895CF92DF92EF92DD
:10086000FF920F931F93CF93DF937C01D62FC72F57
:10087000FC011281058102950F700E940C0C8823E7
:10088000B9F01123A9F08C2F807F803421F080E211
:100890008D0F883068F08091650282FD09C082E08A
:1008A0000E94B50C0E940C0C91E0D82ED92601C0F4
:1008B000D12CCC2EC2948FE0C8228C2D90E08C30AD
:1008C000910508F0CFC1FC01EA5AFF4F0C94F11FCB
:1008D0008C2F807FCF70882311F0C295C07F1123A9
:1008E00099F0CC2309F4AAC180E28D0F883010F072
:1008F000D11104C08C2F0E94160C03C08C2F0E94B3
:10090000260C0E94550C9AC18D2F0E949703CC2370
:1009100009F4A8C180E28D0F883038F1DD2329F178
:100920008C2F0E942C0C24C08C2F807FCF708032A3
:1009300011F0C295C07FDD2319F0D130A1F13DC087
:100940008091650282FF17C0112349F0CC2329F062
:100950008C2F0E94160C0E94550C80E070C180E024
:100960000E949703CC2309F47DC18C2F0E941C0C9C
:100970000E94550C77C1112371F0002341F0013022
:1009800031F40E94360C8C2B0E943E0C6BC10E94ED
:10099000360C8C2B1DC0002319F0013009F462C104
:1009A0000E944B0C25C0112321F0063008F05AC1DB
:1009B0000EC0053008F056C11BC0112361F00023A2
:1009C00031F0F701858180FF39C18F7085838C2FCD
:1009D0000E941F0447C1002359F0D93309F03FC1D9
:1009E000FFEF07EE13E0F15000401040E1F735C192
:1009F0008C2F0E94260436C18C2F86958695837095
:100A000019F0813061F02EC1112321F08D2F9C2F20
:100A1000937002C080E090E00E9406172BC1112362
:100A200021F08D2F9C2F937002C080E090E00E94F7
:100A30001C1720C18D2F112319F00E94791202C0BA
:100A40000E94D4120E944B1315C18C2F837009F0A1
:100A500047C011110BC12D2F229526952770220F0B
:100A6000220F6D2F6F70862F90E0A0E0B0E0022E75
:100A700004C0880F991FAA1FBB1F0A94D2F7D4FF86
:100A800010C04FE050E060E070E004C0440F551F1C
:100A9000661F771F2A95D2F74095509560957095FF
:100AA00003C040E050E0BA01C695C695C3708A0104
:100AB0009B01082B192B2A2B3B2BC901B801C230F3
:100AC00049F058F4C13019F00E942E07CFC00E949F
:100AD0001C07CCC00E944007C9C00E941A07C6C0AC
:100AE000112319F08C2F817001C08695882309F499
:100AF000BDC02D2F229526952770220F220F6D2F16
:100B00006F70862F90E0A0E0B0E0022E04C0880F46
:100B1000991FAA1FBB1F0A94D2F7D4FF10C04FE041
:100B200050E060E070E004C0440F551F661F771F5F
:100B30002A95D2F7409550956095709503C040E096
:100B400050E0BA01C695C695C3708A019B01082B77
:100B5000192B2A2B3B2BC901B801C23049F058F49C
:100B6000C13019F00E94F30781C00E94E1077EC0E6
:100B70000E9405087BC00E94540778C0CF701123E3
:100B800039F08C2F0E947A078D2F0E941F046EC0AF
:100B90008D2F0E9426048C2F0E949B0767C0D23F96
:100BA00021F128F4D03F41F0D13FC1F043C0D33F01
:100BB00019F1D43F79F03EC0112341F0053008F01F
:100BC00051C08C2F8F710E94C0074CC0063008F0B6
:100BD00049C0F7CF8091650282FF18C0112339F018
:100BE0008C2F8F710E947A073DC01123C9F38C2F7F
:100BF0008F710E949B0736C0112329F08C2F8F71B3
:100C00000E9465072FC00E9460072CC0112349F085
:100C1000CF718C2F0E947A0763E08C2F0E949A0C70
:100C200021C081E00E94B50C0230E0F082E00E9419
:100C3000B50C18C0112331F0002391F28D2F0E94C2
:100C4000ED0210C0002399F2D93349F41FEF27EECB
:100C500033E0115020403040E1F700C000008D2FFC
:100C60000E94970388EF8C0D843020F40E94D216E6
:100C70000E948202DD20C9F00E94080C80FD15C090
:100C8000F70112820E94020C0E947A07C7010E949B
:100C900076060E94020CDF91CF911F910F91FF9079
:100CA000EF90DF90CF900C949B07DF91CF911F9135
:100CB0000F91FF90EF90DF90CF9008950F931F93C7
:100CC000CF93DF93EC01688179818A810E94BA0811
:100CD0008C010E9417080E940807B801CE010E94EB
:100CE0002D04DF91CF911F910F910895CF93DF9342
:100CF000EC01988189812B813C81232B31F08F3F3E
:100D000031F481E09F3F19F403C081E001C080E02D
:100D100080FD1DC0CE010E942002811110C00E94E2
:100D20000C0C8823A1F08A81882389F080916502C8
:100D300082FD0DC082E0DF91CF910C94B50CCE0105
:100D40000E945E06CE01DF91CF910C940102DF91EB
:100D5000CF91089580E090E00E94061780E090E037
:100D60000E941C170E94330C0E94550C0E947C1498
:100D70000C944B1380910201909103010E94DE17A5
:100D80000C94AA060E94230C0C94BA0692959F70AC
:100D9000963079F010F4925001C09A50923068F475
:100DA000803F69F018F4883E40F409C0843F29F47C
:100DB00006C0883E20F0813F11F080E0089581E078
:100DC0000895FC01808191810E94AF080E94C606AF
:100DD0000895CF93DF9300D000D01F92CDB7DEB738
:100DE0000F900F900F900F900F90DF91CF9108957B
:100DF000CF93DF9300D000D000D0CDB7DEB72696DA
:100E00000FB6F894DEBF0FBECDBFDF91CF9108952E
:100E1000089508950C9409070C940A070E940C0782
:100E20006093960170939701809398019093990134
:100E30000C94AA060C940E070F931F930091960131
:100E4000109197012091980130919901602B712B9D
:100E5000822B932B1F910F910C940E070F931F93CE
:100E6000009196011091970120919801309199017C
:100E700060237123822393231F910F910C940E07FB
:100E80000F931F9300919601109197012091980163
:100E90003091990160277127822793271F910F9125
:100EA0000C940E070C9409070E945207609392015C
:100EB0007093930180939401909395010C94AA06EA
:100EC00060E070E0CB010C9454070F931F9341E056
:100ED00050E060E070E08A019B0104C0000F111F28
:100EE000221F331F8A95D2F7C901B8011F910F91B4
:100EF0000C9454070F931F9341E050E060E070E0C2
:100F000004C0440F551F661F771F8A95D2F7809142
:100F1000920190919301A0919401B09195018A0161
:100F20009B01082B192B2A2B3B2BC901B8011F91C0
:100F30000F910C9454070F931F9341E050E060E031
:100F400070E004C0440F551F661F771F8A95D2F7C3
:100F50004095509560957095809192019091930184
:100F6000A0919401B09195018A019B010823192356
:100F70002A233B23C901B8011F910F910C945407F8
:100F80000F931F9341E050E060E070E004C0440F15
:100F9000551F661F771F8A95D2F780919201909115
:100FA0009301A0919401B09195018A019B010827BA
:100FB00019272A273B27C901B8011F910F910C94CB
:100FC00054070F931F930091920110919301209168
:100FD000940130919501602B712B822B932B1F91E3
:100FE0000F910C9454070F931F930091920110914D
:100FF0009301209194013091950160237123822304
:1010000093231F910F910C9454070F931F930091FA
:1010100092011091930120919401309195016027E4
:101020007127822793271F910F910C9454070895DD
:10103000990F990F890FE82FE695E695E695877049
:1010400051E001C0550F8A95EAF785E0E89FF0016D
:101050001124E857FE4F20E030E070E04081CB01E2
:10106000022E02C0969587950A94E2F781708195C9
:1010700084278523842781932F5F3F4F25303105B7
:1010800069F70895990F990F890F682F66956695EE
:101090006695982F977085E0689FB001112440E015
:1010A00050E080E0FB01E40FF51FE857FE4F208180
:1010B00030E0092E02C0369527950A94E2F7217098
:1010C0003327042E01C0220F0A94EAF7822B4F5FC8
:1010D0005F4F4530510531F70895BF92CF92DF92AF
:1010E000EF92FF920F931F93CF93DF938C01C090E9
:1010F0009201D0909301E0909401F090950180913D
:10110000960190919701A0919801B0919901C82AF8
:10111000D92AEA2AFB2ACFE1D0E0D701C6010C2E5A
:1011200004C0B695A795979587950A94D2F780FD48
:1011300004C0219790F7B12C07C0BC2EB8018C2FAA
:101140000E949C0F0197A9F38B2DDF91CF911F91E6
:101150000F91FF90EF90DF90CF90BF900895CF93C5
:10116000DF93EC010E946D08BE010E949C0FDF918D
:10117000CF9108951F93CF93DF93EB019091870157
:10118000992321F0CB010E94AF0813C0882349F0B6
:10119000CB010E946D08182F682FCE010E941808FD
:1011A00004C0CB010E944208182FBE01812F0E946B
:1011B0009C0FDF91CF911F9108951F93CF93DF93E1
:1011C000C0919A0116E080919B01C81799F0D0E078
:1011D0001C9FF0011D9FF00D1124E456FE4F40812D
:1011E000518162817381848195810E94F8062196E4
:1011F000C770E9CFDF91CF911F9108954091CC0145
:101200005091CD016091CE017091CF018091D001BC
:101210009091D1010C94F806EF92FF920F931F93D7
:10122000CF93DF938091D10182958F7009F065C0D3
:101230008091CE01882309F460C080919A01F090DA
:101240009B011091CC010091CD016091CF01709173
:10125000D00191E01F3F09F090E0C0910001D091D2
:101260000101292F96E0E92E8F1509F446C061157A
:10127000710521F00F3F21F030E003C031E001C0E3
:10128000322F90E030FD36C0E89EF001E99EF00D6F
:101290001124DF01A456BE4F11963C9111973013D3
:1012A00029C03C91311326C012963C9112973111FE
:1012B00021C013964D915C911497461B570B4C1708
:1012C0005D07C0F48091D1018F7080618093D1015E
:1012D000EF55FE4F80818F70806180838CEC91E0B0
:1012E0000E947606DF91CF911F910F91FF90EF90B2
:1012F0000C94DD0801968770B7CFDF91CF911F91D5
:101300000F91FF90EF9008959F92AF92BF92CF926E
:10131000DF92EF92FF920F931F93CF93DF93CDB79E
:10132000DEB761970FB6F894DEBF0FBECDBF8C015C
:1013300085E0F801DE011D9601900D928A95E1F796
:10134000D8011296EC909091CC01E091CD012091C2
:10135000CF013091D0012115310531F0EF3F31F44B
:1013600081E09F3F19F403C081E001C080E0B82F05
:10137000B1709B2E80FD47C1D8014C9111965C91B4
:1013800011971396AD90BC9014978CECC82E81E009
:10139000D82EF090CE01B501621B730B2091000195
:1013A00030910101FF2009F4D9C08091D101621769
:1013B000730708F095C0282F207F09F052C05E13F4
:1013C00013C0491311C0FE2CE1100EC08F70806154
:1013D0008093D1010E94FE08C6010E94760680918A
:1013E000D101F80185834DC1AB2831F05F3F31F465
:1013F00081E04F3F19F403C081E001C080E080FD2F
:1014000003C081E08E2502C080E090E0F82FF170EB
:10141000FF2E80FF1CC080919A0120919B0136E035
:10142000821709F40BC190E0389FF001399FF00D4D
:101430001124E456FE4F6181561306C060814613A5
:1014400003C06281E61203C001968770E9CFFE2CCB
:10145000EE2009F416C18091D10181608093D10101
:1014600054C05E1306C0491304C0E11002C0F80165
:1014700099C0C8010E94E106882361F1EE2051F174
:101480002091D101822F82958F7090E0029774F0A5
:101490008091CC019091CD0198878F831986BB866E
:1014A000AA862C87CE0107960E94760686E0F80170
:1014B000ACECB1E001900D928A95E1F70E940C0925
:1014C0000E94FE080AC05E1711F1C8010E94E106E1
:1014D00081112CC0C8010E947606FF24F394D1C06C
:1014E000282F207F81F77A2DB98AA88A6E2D8989C5
:1014F0000E94E9068CEC91E00E94760686E0D60117
:101500001D928A95E9F70E94FE08F12CBAC0491392
:10151000DCCFE110DACFF8018583C8010E9476069E
:1015200086E0D6011D928A95E9F7ABC0EE2091F2D4
:101530002091D101822F82958F7090E002970CF458
:10154000B5CF8091CC019091CD019A8389831B8284
:10155000BD82AC822E83CE010196A6CF621773079F
:1015600008F044C0FE2CEE2009F4B4CF5E1330C066
:1015700049132EC02091D10120FD21C0822F8295D8
:101580008F70482F50E041155105C9F0F8012583AF
:101590004F30510541F08F5F982F9295907F822FA9
:1015A0008F70892B8583C8010E94760686E0F8013A
:1015B000ACECB1E001900D928A95E1F73CC086E079
:1015C000F801ACECB1E001900D928A95E1F759C0B9
:1015D000C8010E94E106811169CF8091D10181602B
:1015E0008093D101C8010E9476064BC07A2DB98A3A
:1015F000A88A6E2D89890E94E90686E0D6011D928F
:101600008A95E9F718C0EE2009F464CFC8010E945A
:10161000E106F82E882309F45DCF86E0F801ACECF2
:10162000B1E001900D928A95E1F78CEC91E00E9477
:10163000E7020E940C090E94FE0823C04D875E87C6
:101640008D859E850E94AF08292F22952F7022300C
:1016500028F49F7039F0811105C00BC0243028F4A4
:101660009F7049F4805E883020F0C8010E947606A1
:101670009F2CF92C06C0D80115969C91907F91F76C
:10168000F8CF8F2D61960FB6F894DEBF0FBECDBF99
:10169000DF91CF911F910F91FF90EF90DF90CF904E
:1016A000BF90AF909F9008951F93CF93DF93CDB7D6
:1016B000DEB72C970FB6F894DEBF0FBECDBF4F83B9
:1016C000588769877A878B879C87CE0107960E9407
:1016D00084098823D1F09F8188852A853B85232B27
:1016E00031F08F3F31F481E09F3F19F403C081E076
:1016F00001C080E080FD47C04F81588569857A85AB
:101700008B859C850E94F8063EC086E0FE013796D8
:10171000DE01119601900D928A95E1F7FF81E8852F
:101720006A857B856115710531F0EF3F31F481E009
:10173000FF3F19F403C081E001C080E080FD23C0B9
:1017400020919B0130E0C901019687709927409153
:101750009A0150E084179507F1F1F983EA837D83BC
:101760006C8396E0929FD001939FB00D1124A456F4
:10177000BE4FFE01319601900D929A95E1F780934C
:101780009B010E94DD0816E080919A0190919B01D7
:10179000891771F1189FC001112484569E4F0E9431
:1017A0008409882329F1E0919A011E9FF0011124F8
:1017B000E456FE4F4081518162817381848195811D
:1017C0000E94F80680919A0190E00196877099270F
:1017D00080939A01D9CF0E94C20610929B01109269
:1017E0009A01ECECF1E086E0DF011D928A95E9F7C1
:1017F0002C960FB6F894DEBF0FBECDBFDF91CF9110
:101800001F9108958091F20185958595859508959C
:101810008091F201877008959091F201977081E0B4
:1018200009F480E0089580911502089590911502C1
:10183000892B809315020895809590911502892334
:101840008093150208951092150208959091140244
:10185000892B809314020895809590911402892316
:101860008093140208951092140208958091F30158
:10187000089508950C94390C0C943A0C90916502DB
:1018800092FD08C09091F301981721F08093F30125
:101890000C943C0C08958091F301882329F0109258
:1018A000F30180E00C943C0C0895CF93DF93E0911A
:1018B0000201F0910301809115028083E091020101
:1018C000F0910301908180911402892B8083809193
:1018D000F301882381F0E0910201F09103019081EE
:1018E000892B808380910201909103010E9432171D
:1018F00081110E944B0CC0910201D091030140E282
:1019000050E062ED71E0CE010E940B20892B69F05E
:1019100080E2FE01A2EDB1E001900D928A95E1F71F
:10192000CE01DF91CF910C94DE16DF91CF91089517
:101930000C94390C9091650292FD10C098E0899F3B
:1019400090011124262B2093F2010E947A078091A6
:10195000F2018595859585950C94980C0C947A07E1
:101960001092F20180E00C94980C2091F201809585
:1019700082238093F201982F977099F430E0482FDA
:10198000082E000C550B2417350759F0909165026D
:1019900092FD07C08595859585950E949B070C94BF
:1019A000B00C08959091650292FB222720F9281728
:1019B00069F080FB92F990936502809164029091A6
:1019C00065020E941A0D82E00C94B50C0895809176
:1019D000650282FB882780F991E089270C94D20C5C
:1019E00081E00C94D20C80E00C94D20C80E090E06A
:1019F0000E94202021E0893E9E4F09F020E0822FA6
:101A0000089582E090E00C94182083E090E00C941C
:101A10001820CF9384E090E00E941820C82F82E223
:101A200090E00E9418202C2F30E0A901582BCA0109
:101A3000CF910895CF93C92F682F84E090E00E9442
:101A400026206C2F82E290E0CF910C942620AB01EF
:101A5000BC018FE090E00C943820AB01BC0183E125
:101A600090E00C94382060E070E0CB010C942D0DD8
:101A700060E070E0CB010E94270D0C94330D69EEFD
:101A80007EEF80E090E00E94442060E082E090E001
:101A90000E94262060E083E090E00E9426201092C1
:101AA000960110929701109298011092990160E0AE
:101AB00084E090E00E94262060E082E290E00E94B4
:101AC000262060E085E090E00E94262060E086E02D
:101AD00090E00E9426206FEF87E090E00E94262091
:101AE00040E050E0BA0188E090E00E94382060E0D9
:101AF0008DE090E00E94262040E050E0BA0188E1AD
:101B000090E00E94382060E087E190E00E9426206B
:101B100040E050E0BA018CE190E00E94382060E0A3
:101B200070E080E290E00E94442040E050E0BA0182
:101B300088E190E00E9438200C94380D0C943F0D01
:101B4000682F8EE090E00C9426200E9497186093F6
:101B50001E0270931F0280932002909321026093D3
:101B60001A0270931B0280931C0290931D02089529
:101B700085B7806885BF85B7806885BF089581E097
:101B800008950C94BF0D08950C94C30D0C94C30DCF
:101B90000C94C60D0C94C30D0C94CA0D0C94C30D7B
:101BA0000E94B80D88E790E10E94C8160E94CE0DF1
:101BB0000C94CC0D0E94C40D0C94C30D0E947B109C
:101BC0000C9481020E9482180E9455110E94DE0D21
:101BD0000C94C80D8F929F92AF92BF92CF92DF92DA
:101BE000EF92FF920F931F93CF93DF93CDB7DEB7A2
:101BF0002A970FB6F894DEBF0FBECDBF0E946A11C0
:101C0000982E81110E94A50D86E1A82E82E0B82EA3
:101C100000E010E0802E802F0E949F10D82EF5014A
:101C2000C1905F01C826B1F40F5F1F4F043011054A
:101C300089F78FEF89838A831B820E948B188160CA
:101C4000782F9D838C8349815A816B818D810E947D
:101C50009D022FC08091220281FD0E94A510E12CDF
:101C6000FF24F3948C2D8F21F1F00E94C10D882365
:101C700099F0EE828F82DF2081E009F480E088878E
:101C80000E948B188160782F9A8789874E815F81A7
:101C900068858A850E949D02F801EA5EFD4F808179
:101CA000F826F08206C0E394FF0CF4E0EF12DACFDE
:101CB000BBCF81E0911001C080E02A960FB6F89466
:101CC000DEBF0FBECDBFDF91CF911F910F91FF906F
:101CD000EF90DF90CF90BF90AF909F908F9008953E
:101CE0000E94EA0D0E9469130C949202CF93DF9335
:101CF0000E94A10FEC01811521E5920708F045C073
:101D0000811530E5930708F094C0883E910528F5C9
:101D1000803E910508F0F8C0883A910570F4853A44
:101D2000910508F07CC08130910509F475C008F474
:101D3000E8C0049708F0E8C0E4C08F3B910508F0C4
:101D4000E0C0C85AD0E0CC0FDD1FC65BDE4F099063
:101D5000D881C02DCE019464D8C0811540E294078B
:101D600058F4811551E0950708F0CEC08D3E9105DD
:101D700008F4C7C09065C9C0C11580E4D80708F44D
:101D8000C0C0DF70CE01906AC0C0811525E5920702
:101D9000A8F4811534E5930708F095C0811543E553
:101DA000940708F07BC0811552E5950708F061C0E3
:101DB000D82FCC27CE01816F906AA7C0C11589E5C5
:101DC000D807A0F4C11528E5D20708F082C0C115D4
:101DD00036E5D30708F095C08C2F0E9435108F711F
:101DE00090E0D82FCC27CE0190628FC0C1154AE574
:101DF000D40708F474C0CE0190568115904208F0C3
:101E000080C08D2F8F710E943510DD27D0628F71B9
:101E1000AE01582BCA0179C081E090E076C0C55A66
:101E2000D0E0C858DE4F8881C82FD0E0CE01906442
:101E30006CC074E0969587957A95E1F7282F23700A
:101E40003C2F337081E090E002C0880F991F3A95D3
:101E5000E2F79C68AC01522B9A019C2F9F709695DB
:101E6000969550E2959FE0011124C9018C2B9D2B82
:101E70004CC08370992721E030E002C0220F331F4D
:101E80008A95E2F79C2F9695969580E2989FE001BF
:101E90001124C22BD32BCE019C6837C083709927A5
:101EA00021E030E002C0220F331F8A95E2F79C2F19
:101EB0009695969540E2949FE0011124C22BD32B76
:101EC000CE019A6822C0D82FCC27CE01846F906AA9
:101ED0001CC0DC2FCC27CE01806F906A16C08C2FDF
:101EE0008F700E94351094E0D695C7959A95E1F7CA
:101EF000CF70D0E0DC2FCC27D0699E01282BC90100
:101F000004C080E090E001C0CE01DF91CF91089540
:101F1000E72FF0E094E0899FE00DF11D1124EE0F12
:101F2000FF1FEE0FFF1FE60FF11DEE0FFF1FE85220
:101F3000FF4F8591949108950E94880F0E94760E1C
:101F400008958238910569F1B0F48133910509F45F
:101F50006DC048F48932910509F463C08A32910555
:101F600009F469C008958533910509F455C0893392
:101F70009105B9F00895833E910569F138F4803EEA
:101F80009105B1F0823E910509F10895863E9105D3
:101F9000A9F1873E9105B9F1843E910509F064C02D
:101FA00023C02091640220FD4FC021FD4DC0089543
:101FB0008091640280FD44C08091650280FF44C02E
:101FC0008091640284FD42C083EE4DC08091640222
:101FD00082FF38C0F5CF8091640282FD33C08091CA
:101FE000650280FD31C0ECCF8091650281FF32C077
:101FF0008091640284FD2AC087EE35C0809164021E
:1020000083FF26C0F5CF8091640283FD21C08091BB
:10201000650281FD1FC0ECCF8091640285FD1CC06C
:102020001DC08091640285FD19C016C080916402B4
:1020300086FD16C017C08091640286FD13C010C0D3
:1020400089E311C082EE0FC080EE0DC080E00BC0AE
:1020500086EE09C084EE07C089E205C085E303C0AF
:102060008AE201C081E390E008959091640292FFBA
:102070000DC0282F2871283019F4877F846006C08E
:10208000282F2471243011F48B7F886093FF0DC0BA
:10209000282F2871283119F4877E846106C0282FE3
:1020A0002471243111F48B7E88612091650220FF18
:1020B0000DC0382F3871383019F4877F816006C021
:1020C000382F3171313011F48E7F886021FF0DC0BF
:1020D000282F2871283119F4877E816106C0282FA6
:1020E0002171213111F48E7E886194FD877E0895DF
:1020F00080E0089508950E94F60C811102C00E94AC
:102100009E0D0E94010D809322020E94090D909362
:102110006502809364020E947A100E94050D682F68
:1021200070E080E090E00E941A0760919201709147
:10213000930180919401909195010C945207E82F9E
:10214000F0E0E659FD4F80810895089580EA8A9570
:10215000F1F7089500C008950C94A61008950C940A
:10216000AE100C94AF100C94B501F894E82FE295E2
:10217000EF70F0E031A1282F2F7081E090E001C0D6
:10218000880F2A95EAF7982F9095932391A392A10F
:10219000892B82A3789408950F931F93CF93DF9395
:1021A000CBE7D1E089918F3F11F00E94B51081E01B
:1021B000CF37D807B9F7CFE7D1E003E811E089912D
:1021C0008F3F11F00E94B5100C171D07C1F7DF916A
:1021D000CF911F910F910895EF92FF920F931F934C
:1021E000CF93DF93C62FD0E0C558DE4F28812F3F15
:1021F00009F454C0042F162F7C01F894E22FE295C5
:10220000EF70F0E081A1422F4F7021E030E001C07B
:10221000220F4A95EAF7822B81A382A120952823D9
:1022200022A378940E94AA106FE771E0F701A7013A
:102230004C5F5F4FF12C302F3095DB012D91BD01AC
:102240002F3FB1F0822F82958F7090E0DC01909645
:102250008C9190E02F7002C0959587952A95E2F7B2
:1022600080FD06C08081802B8083FF24F39403C00F
:102270008081832380833196E417F507F1F6888106
:102280008F3F11F00E94B5106F2D812FDF91CF91FC
:102290001F910F91FF90EF900C94AC10DF91CF91B4
:1022A0001F910F91FF90EF9008950E94CC1084E051
:1022B000EAE6F2E0DF01982F1D929A95E9F7E6E64B
:1022C000F2E0DF011D928A95E9F784E00E94B111E6
:1022D0000C940C020F931F93CF93DF9300D000D088
:1022E000CDB7DEB719821A821B821C8210E001E092
:1022F000402F612FCE0101960E94EC101F5F000F4E
:102300001430B1F744E050E0BE016F5F7F4F86E6C6
:1023100092E00E940B2011E0009709F410E0892B55
:1023200061F089819A81AB81BC8180936602909330
:102330006702A0936802B0936902212F44E06AE625
:1023400072E086E692E00E94B2110E940E02812F96
:102350000F900F900F900F90DF91CF911F910F91E1
:1023600008950895FF920F931F93CF93DF938C01ED
:10237000F62ED72FC42F222349F081E08093250227
:102380000E948B189093240280932302809125024F
:102390008823C1F080912302909124020E94A31807
:1023A000059780F0EF2DFD2FD8014C2F50E0CD0187
:1023B000801B910B841795071CF48D918193F7CFA7
:1023C00010922502DF91CF911F910F91FF900895F8
:1023D0000E94A31A0E94E20D0C94AF1A0E94B31A35
:1023E0000E94700E0C94CD1A0E9429180E948A1A1D
:1023F0000E94D00D0E94E8110E94EE110E94DA0D99
:10240000FBCF80912C0280FF06C06091090170E033
:10241000660F771F26C081FF04C06091090184E028
:1024200005C082FF07C06091090188E0689FB00184
:10243000112417C090912B029923D1F060910801CB
:10244000961788F72091090188E0289F90011124B0
:10245000929FA001939F500D112470E0CA010E9429
:10246000DD1F6038710540F46115710519F406C06F
:1024700068E070E0862F08958FE7089581E0089561
:1024800080912C0280FF08C06091050170E0759575
:1024900067957595679521C081FF06C0609105011C
:1024A00070E07595679519C082FF04C060910501C1
:1024B00070E010C090912A02992399F06091040174
:1024C0009617A0F780910501899FC001112470E043
:1024D0000E94DD1F6038710540F46115710519F423
:1024E00006C061E070E0862F08958FE7089581E0CF
:1024F00008958D3E21F40E940112819504C08E3E04
:1025000029F40E9401128093300208958F3E21F435
:102510000E940112819504C0803F29F40E9401129B
:1025200080932F020895893F19F40E94401205C03C
:102530008A3F31F40E9440128195809331020895C0
:102540008B3F21F40E944012819504C08C3F29F4F6
:102550000E9440128093320208959FE0980F9830B5
:1025600078F421E030E0A90102C0440F551F9A958C
:10257000E2F7CA0190912E02892B80932E020895D2
:102580008D3F21F480912C0281600BC08E3F21F49D
:1025900080912C02826005C08F3F29F480912C022B
:1025A000846080932C0208958D3E39F4909130021E
:1025B00097FF35C01092300259C08E3E29F4909199
:1025C00030021916BCF32BC090912F028F3E29F4D4
:1025D00097FF25C010922F0249C0803F19F41916A9
:1025E000CCF31DC090913102893F29F41916BCF437
:1025F000109231023BC08A3F19F497FF10C0F8CF08
:102600008B3F39F49091320297FF09C01092320249
:102610002DC08C3F21F4909132021916BCF39FE03B
:10262000980F983080F421E030E0A90102C0440FF7
:10263000551F9A95E2F7CA01809590912E02892341
:1026400080932E0213C08D3F21F480912C028E7F47
:102650000BC08E3F21F480912C028D7F05C08F3FEF
:1026600029F480912C028B7F80932C0280912F0281
:10267000811106C080913002811102C010922B029C
:1026800080913102811106C080913202811102C015
:1026900010922A0208950E948B1820912F02211176
:1026A00004C020913002222321F0909329028093CC
:1026B000280220913102211104C0209132022223EC
:1026C00021F090932702809326028DE292E00C94F1
:1026D000F816EF92FF920F931F93CF93DF9300D0E2
:1026E00000D000D0CDB7DEB786E0EDE2F2E0DE014B
:1026F000119601900D928A95E1F7E0902F02F090EB
:102700003002009131021091320210922F02109289
:1027100030021092310210923202E11003C0FF2009
:1027200009F45DC080912802909129020E94A318AB
:10273000AC0190912B02992339F020910A0130E0ED
:102740002417350758F04BC020910B018AE0289FD1
:10275000900111242417350718F041C09F3F19F04C
:102760009F5F90932B02EE2061F00E9401121E14D5
:1027700014F09FEF01C091E0989F902D1124909349
:102780002F02FF2061F00E9401121F1414F09FEF2E
:1027900001C091E0989F902D1124909330023091C8
:1027A0002F023323E1F0209130022223C1F045EBC8
:1027B0003403C0011124992319F090932F0203C010
:1027C00081E080932F0235EB2303C001112499236C
:1027D00019F09093300203C081E080933002011120
:1027E00003C0112309F45DC0809126029091270255
:1027F0000E94A318AC0190912A02992339F02091EC
:10280000060130E02417350758F04BC0209107012E
:102810008AE0289F900111242417350718F041C041
:102820009F3F19F09F5F90932A02002361F00E945E
:102830004012101614F09FEF01C091E0989F902D68
:10284000112490933102112361F00E94401211165D
:1028500014F09FEF01C091E0989F902D1124909368
:102860003202309131023323E1F0209132022223EF
:10287000C1F045EB3403C0011124992319F0909362
:10288000310203C081E08093310235EB2303C001A4
:102890001124992319F09093320203C081E08093B0
:1028A000320280912F0281110BC080913002811180
:1028B00007C080913102811103C0809132028111E1
:1028C0000E944B13EB82FC820D831E8386E0FE0187
:1028D0003196ADE2B2E001900D928A95E1F726962D
:1028E0000FB6F894DEBF0FBECDBFDF91CF911F9121
:1028F0000F91FF90EF900895EDE2F2E086E0DF01A6
:102900001D928A95E9F710922B0210922A021092DA
:102910002C020895CF93DF93EC01FB018281882381
:1029200009F43CC1C430FDE5DF0760F4CB3F9CE512
:10293000D90788F49E0122503C452431310508F026
:102940002EC109C0C236EDE5DE0729F0C63AFDE525
:10295000DF0709F024C10E94090D9093650280935E
:102960006402C1318CE5D80709F4C6C008F042C042
:10297000C930ECE5DE0709F49BC000F5C5308CE5F5
:10298000D80709F485C078F4C330ECE5DE0709F414
:1029900078C008F07AC0C230DC4509F0F5C08091FB
:1029A00064028160EFC0C7309CE5D90709F478C0A4
:1029B00008F07AC0809164028061E4C0CD30FCE50B
:1029C000DF0709F487C058F4CB309CE5D90709F438
:1029D00079C008F07BC08091640288606FC0CF30FE
:1029E000FCE5DF0709F480C008F082C08091640232
:1029F000877FC8C0CE3F9CE5D90709F471C000F5B8
:102A0000C531FCE5DF0709F485C068F4C3319CE5F6
:102A1000D90709F475C008F095C00E94C2068091DC
:102A200064028F77AFC0CC3FFCE5DF07A9F108F067
:102A300054C0CB3FDC4509F0A7C08091650240C07F
:102A4000C230EDE5DE0709F489C058F4C1158DE503
:102A5000D80709F45AC008F069C080916502826005
:102A60002FC0C236EDE5DE0709F47CC0C63AFDE5AD
:102A7000DF0709F481C0C330DD4509F085C080E07F
:102A80006EC08091640282607DC08091640216C035
:102A900080916402886076C08091650282604FC038
:102AA0008091640280626EC08091640280646AC01A
:102AB0000E94C20680916402806864C0846062C023
:102AC00081603DC0809164028E7F5CC08091640211
:102AD0008D7F58C08091640216C08091650218C035
:102AE000809165028D7F2BC0809164028F7E4AC0E9
:102AF000809164028F7D46C0809164028F7B42C0CA
:102B000080916402877F8B7F3DC0809165028D7FBD
:102B10008E7F15C08091640282FB222720F991E00C
:102B2000922790FB82F990FB83F92CC0809165027B
:102B3000982F909591708E7F892B90FB81F98093CF
:102B4000650222C00E94C2068091640287FB222790
:102B500020F991E0922790FB87F914C081E00E9450
:102B6000A00D12C08091640284FB222720F991E01D
:102B7000922790FB84F906C080916402982F90956B
:102B800090FB80F9809364028091640290916502C9
:102B90000E941A0D0E94C20680E001C081E0DF9110
:102BA000CF910895CF93DF9386319C4541F5EB019A
:102BB0000E94130C982F8A81209102013091030109
:102BC000882379F09A7A81E009F480E080933302D7
:102BD000911102C069E201C065E3C9010E94C817F2
:102BE0000AC080913302811102C069E201C065E32D
:102BF000C9010E94D3170E94550C80E001C081E0FA
:102C0000DF91CF9108950F931F93CF93DF93C42F3C
:102C1000D22FFC0182818823C9F0409336020E94A2
:102C20008B18909335028093340280E28C0F8830A9
:102C300008F057C0C77081E001C0880FCA95EAF755
:102C4000DF91CF911F910F910C941F048091360258
:102C5000481330C080913402909135020E94A3182D
:102C6000883C910538F510E21D0FCD17B9F080E2D0
:102C70008C0F883040F4C77081E001C0880FCA957E
:102C8000EAF70E942604183028F581E09D2F9770FE
:102C900001C0880F9A95EAF70E941F04802F0E94B6
:102CA00016041830F0F4D77081E001C0880FDA956F
:102CB000EAF70AC080E28C0F883098F4C77081E090
:102CC00001C0880FCA95EAF7DF91CF911F910F914C
:102CD0000C942604802FDF91CF911F910F910C94BB
:102CE0001604DF91CF911F910F9108950F939C01CE
:102CF000CB01243F4CE5340731F188F4293DFCE554
:102D00003F07D9F02A3D4CE5340779F1283D3C4591
:102D1000A9F506E221EE41EE68ED7CE52BC0263FE9
:102D2000FCE53F07E1F0A8F0273F3C4539F507E215
:102D300025EE46EE67EF7CE51DC007E225EE45EE89
:102D400069ED7CE517C006E221EE40EE64EF7CE51C
:102D500011C007E225EE44EE65EF7CE50BC006E20C
:102D600021EE42EE66EF7CE505C008E221E045EE8B
:102D70006AED7CE50E94031680E008C0FC018281B8
:102D8000882319F01092360201C081E00F91089556
:102D90009093850180938401089590933C028093E1
:102DA0003B020895E0913B02F0913C02309721F004
:102DB0000190F081E02D099480E00895E0913B02BC
:102DC000F0913C02309799F020911801222359F09C
:102DD0002091640227FF07C0DC012C9111962C93EF
:102DE000119726E02C930280F381E02D0994089539
:102DF000E0913B02F0913C02309739F022E0DC0197
:102E00002C930480F581E02D0994089520913902D6
:102E100030913A022817390771F090933A02809363
:102E20003902E0913B02F0913C02309721F006809C
:102E3000F781E02D099408952091370230913802EE
:102E40002817390771F09093380280933702E09188
:102E50003B02F0913C02309721F00084F185E02D97
:102E600009940895FC01329680911801882331F06D
:102E70008091640287FF02C09EE101C096E080E07D
:102E8000915028F021912223D9F38F5FF9CF089533
:102E9000662351F1209118012223E9F02091640268
:102EA00027FF19C0462F4695469546954E31E0F4CA
:102EB000677021E030E002C0220F331F6A95E2F70D
:102EC000FC01E40FF11D828190E02823392381E089
:102ED000232B69F409C0FC013296089621916217F0
:102EE00029F0E817F907D1F780E0089581E0089507
:102EF0009C01FC0132969FEF80E04191461789F0DA
:102F00009F3F19F4411101C0982F8F5F8630A9F7B8
:102F10009F3F39F0F901E90FF11D97FDFA956283A2
:102F2000089508959C012A5F3F4FFC01428146139A
:102F300001C01282019682179307B9F70895262FD0
:102F40002695269526952E3168F4FC01E20FF11D99
:102F5000677021E030E001C0220F6A95EAF78281B4
:102F6000282B22830895262F2695269526952E31E7
:102F700070F4FC01E20FF11D677021E030E001C048
:102F8000220F6A95EAF720958281282322830895EB
:102F900020911801222329F02091640227FD0C942E
:102FA0009F170C94781720911801222329F0209163
:102FB000640227FD0C94B3170C949217209118010A
:102FC000FC013296222331F08091640287FF02C017
:102FD0008EE101C086E0DF011D928A95E9F7089530
:102FE00008950C94F01783E080933D020C94F11740
:102FF000811102C081E001C082E080933D020C9407
:10300000F1170C94F81781E080933D020C94F117AE
:103010000C94031808950C940A180C940B180C9433
:103020000A180C940A180C940A18CF930E941118CD
:103030000E946A110E940F18C0E08C2F0E949F10FE
:10304000811104C0CF5FC430C1F701C081E0CF91CE
:10305000089508951F920F920FB60F9211248F9327
:103060009F93AF93BF9380913E02811113C08091D3
:103070006E0290916F02A0917002B0917102419620
:10308000A11DB11D80936E0290936F02A0937002F8
:10309000B0937102BF91AF919F918F910F900FBE2E
:1030A0000F901F90189580917602843031F10E9424
:1030B000720210923E0220E488E190E00FB6F8948C
:1030C000A895809360000FBE2093600083B7817F36
:1030D000846083BF83B7816083BF7894889583B70A
:1030E0008E7F83BF0FB6F894A895809160008861A9
:1030F00080936000109260000FBE08950E94C20687
:103100000C94760282E084BD93E095BD9AEF97BD62
:1031100080936E0008952FB7F89480916E0290917D
:103120006F02A0917002B09171022FBF08952FB766
:10313000F89460916E0270916F028091700290918C
:1031400071022FBF08959C014FB7F89480916E02D1
:1031500090916F02A0917002B09171024FBF821BDB
:10316000930B089578941F920F920FB60F9211242B
:103170008F939F93AF93BF9380916E0290916F0254
:10318000A0917002B09171020196A11DB11D8093B2
:103190006E0290936F02A0937002B0937102BF9180
:1031A000AF919F918F910F900FBE0F901F90189528
:1031B00081E08093E00080E28093D8001092C90003
:1031C0008FE19EE40197F1F700C0000087E090EBEB
:1031D000DC0180937F0290938002A0938102B093E0
:1031E00082029CE088E10FB6F894A8958093600075
:1031F0000FBE90936000FFCF809162020895089502
:1032000022E02093E9002FEF3091E800215035FDB6
:1032100006C035ED3A95F1F700002111F5CF209168
:10322000E80025FF0BC040E050E066E070E00E943F
:103230003F1B8091E8008E778093E8000895CF933C
:10324000DF9320911801222339F02091640227FF97
:1032500003C060E222E002C068E021E02093E900C0
:103260002FEF3091E800215035FD06C035ED3A953D
:10327000F1F700002111F5CF2091E80025FF1DC0D6
:10328000EC0180911801811105C040E050E068E038
:1032900070E003C070E040E050E0CE010E943F1BB0
:1032A0008091E8008E778093E80080E2FE01A2E43E
:1032B000B2E001900D928A95E1F7DF91CF910895E8
:1032C00080933F02709341026093400280917602A6
:1032D000843001F582E08093E9008FEF9091E8005F
:1032E000815095FD06C095ED9A95F1F7000081118A
:1032F000F5CF8091E80085FF0DC040E050E063E02D
:1033000070E08FE392E00E943F1B8091E8008E778F
:103310008093E8000895BC0184E00C946019BC011E
:1033200083E00C94601980917502811109C00E949C
:10333000D01C0E942D1D8091E20084608093E200E9
:1033400008951092750208950C9408186091720205
:1033500081E0611101C080E00C94F3179091760236
:1033600081E0943009F080E0609172020C94F817CB
:1033700042E061EC81E00E94491C42E261EC82E0A3
:103380000E94491C9091760281E0943009F080E01F
:10339000609172020C94011880917802833009F4D4
:1033A00061C030F4813071F0823009F49AC0089520
:1033B0008A3009F486C08B3009F46CC0893009F07A
:1033C000A8C020C080917702813A09F0A2C0809104
:1033D000E800877F8093E80080917B0290917C02D7
:1033E000892B21F460E282E492E003C060E080E097
:1033F00090E070E00E948A1B8091E8008B778093B8
:10340000E800089580917702813209F082C08091AE
:103410007B0290917C02029708F07BC08091E800CB
:10342000877F8093E8008091E80082FD05C080914D
:1034300076028111F8CF6DC02091F3008091F200E7
:1034400090E0922B029731F48091F100813011F0DD
:10345000863021F48091F100809362028091E8002F
:103460008B7753C080917702813A09F052C08091E6
:103470007B0290917C02892B09F04BC08091E8007F
:10348000877F8093E8008091E80080FFFCCF8091E7
:10349000180136C0809177028132D9F580917B0284
:1034A00090917C02892BA9F58091E800877F809319
:1034B000E8000E947E1C80917902809318010C9490
:1034C000C20680917702813221F58091E800877FE2
:1034D0008093E8000E947E1C80917A0280936302B0
:1034E000089580917702813AA1F48091E800877F66
:1034F0008093E8008091E80080FFFCCF8091630218
:103500008093F1008091E8008E778093E8000C941E
:103510007E1C089584B7877F84BF0FB6F894A89562
:1035200080916000886180936000109260000FBEFF
:1035300090E080E80FB6F89480936100909361006A
:103540000FBE0C9403180E94D01C0E942D1DE2EEA9
:10355000F0E080818460808378940C94C21F8CE0BA
:1035600091E00C94CD16809176028530A9F480917B
:103570007602853079F40E94531880917402882372
:10358000B1F30E941518882391F30E94291B0E9411
:10359000C206EDCF0C947E18089508950C94D01AAD
:1035A000292F332723303105C9F060F4213031054C
:1035B00081F02230310509F044C08BE390E020E532
:1035C00031E043C021323105E1F02232310549F1C9
:1035D00038C082E190E02BE831E037C09927813094
:1035E000910549F028F0029761F5E8E1F1E005C0A6
:1035F000ECE4F1E002C0ECE2F1E0849190E09F01A4
:1036000024C06115710541F061307105D1F489E084
:1036100090E02BE731E019C089E090E022E631E04C
:1036200014C06115710541F06130710551F486EBEC
:1036300090E02DE931E009C080E490E023E532E03C
:1036400004C080E090E020E030E0FA013183208384
:10365000089580E189BD82E189BD09B400FEFDCFF6
:103660008091D8008F7D8093D8008091E0008260A7
:103670008093E0008091E00081FDFCCF0895CF921F
:10368000DF92EF92FF920F931F93CF93DF93EC01A2
:103690008B017A010E949D1C811133C0E114F10459
:1036A00039F0F70180819181081B190BC80FD91FD0
:1036B000C12CD12C0115110519F18091E80085FD6F
:1036C00016C08091E8008E778093E800E114F10441
:1036D00049F0F70180819181C80ED91ED182C08244
:1036E00085E00FC00E949D1C882321F30AC08991A8
:1036F0008093F10001501109FFEFCF1ADF0ADACFF2
:1037000080E0DF91CF911F910F91FF90EF90DF90BC
:10371000CF90089520917D0230917E0226173707C1
:1037200048F06115710539F42091E8002E77209357
:10373000E80001C0B901FC0120E06115710579F1D3
:10374000809176028823F1F18530F1F18091E800D3
:1037500083FD3CC08091E80082FD2EC08091E8008E
:1037600080FFEBCF2091F3008091F20090E0922B4C
:103770006115710551F08830910538F4219120933D
:10378000F100615071090196F3CF21E0089709F02B
:1037900020E08091E8008E778093E800CECF211161
:1037A000CFCF0AC080917602882361F0853061F026
:1037B0008091E80083FD0AC08091E80082FFF2CF8B
:1037C00080E0089582E0089583E0089581E00895FF
:1037D00020917D0230917E022617370748F061154F
:1037E000710539F42091E8002E772093E80001C09C
:1037F000B901FC0120E06115710591F1809176021B
:10380000882309F440C0853009F43FC08091E80066
:1038100083FD3DC08091E80082FD2FC08091E800CB
:1038200080FFE9CF2091F3008091F20090E0922B8D
:103830006115710559F08830910540F42491209369
:10384000F1003196615071090196F2CF21E008979D
:1038500009F020E08091E8008E778093E800CBCFDC
:103860002111CCCF0AC080917602882361F0853087
:1038700061F08091E80083FD0AC08091E80082FF3A
:10388000F2CF80E0089582E0089583E0089581E01A
:103890000895982F973068F59093E900981739F0BC
:1038A0007091EC002091ED005091F00003C0242FA6
:1038B000762F50E021FD02C09F5FECCF3091EB00EE
:1038C0003E7F3093EB003091ED003D7F3093ED0073
:1038D0003091EB0031603093EB007093EC0020935B
:1038E000ED005093F0002091EE0027FDE5CF80E041
:1038F00008958F708093E90081E0089580917702A8
:1039000087FF11C08091E80082FD05C0809176029A
:103910008111F8CF11C08091E8008B770BC08091A6
:103920007602882349F08091E80080FFF8CF8091EB
:10393000E8008E778093E80008952091E4003091AC
:10394000E50095E64091EC00842F817040FF23C094
:103950008091E80080FD1DC080917602882399F057
:10396000853099F08091EB0085FD11C04091E40015
:103970005091E5002417350729F3915011F09A0171
:10398000E1CF84E0089582E0089583E0089581E026
:10399000089580E008954091E80042FFDDCF08954A
:1039A0000E943E1D0E94461DE0EEF0E08081816095
:1039B0008083E8EDF0E080818F77808319BCA7EDEC
:1039C000B0E08C918E7F8C9380818F7E808310926B
:1039D000750208950F931F93CF93DF930E943E1DAE
:1039E0000E94461DC8EDD0E088818F77888388814A
:1039F0008068888388818F7D888319BC10927602C5
:103A000010927202109274021092730200EE10E093
:103A1000F80180818B7F808388818160888342E088
:103A200060E080E00E94491CE1EEF0E080818E7F42
:103A30008083E2EEF0E08081816080838081886015
:103A40008083F80180818E7F808388818061888374
:103A5000DF91CF911F910F910895E8EDF0E0808103
:103A60008F7E8083E7EDF0E080818160808384E059
:103A700082BF81E0809375020C94EA1CE8EDF0E0CF
:103A800080818E7F80831092E20008951092DA0088
:103A90001092E10008951F920F920FB60F92112419
:103AA0002F933F934F935F936F937F938F939F9346
:103AB000AF93BF93EF93FF938091E10082FF0BC020
:103AC0008091E20082FF07C08091E1008B7F8093AC
:103AD000E1000E94C11F8091DA0080FF1FC0809129
:103AE000D80080FF1BC08091DA008E7F8093DA00BF
:103AF0008091D90080FF0DC080E189BD82E189BD40
:103B000009B400FEFDCF81E0809376020E949319F4
:103B100005C019BC109276020E94A1198091E100A3
:103B200080FF19C08091E20080FF15C08091E20003
:103B30008E7F8093E2008091E20080618093E200BA
:103B40008091D80080628093D80019BC85E0809372
:103B500076020E94A6198091E10084FF30C0809116
:103B6000E20084FF2CC080E189BD82E189BD09B4F7
:103B700000FEFDCF8091D8008F7D8093D80080918A
:103B8000E1008F7E8093E1008091E2008F7E809340
:103B9000E2008091E20081608093E20080917202F5
:103BA000882311F084E007C08091E30087FD02C004
:103BB00081E001C083E0809376020E94AE1980917B
:103BC000E10083FF29C08091E20083FF25C080913E
:103BD000E100877F8093E10082E08093760210927B
:103BE00072028091E1008E7F8093E1008091E2007B
:103BF0008E7F8093E2008091E20080618093E200FA
:103C000042E060E080E00E94491C8091F000886002
:103C10008093F0000E94A419FF91EF91BF91AF91A2
:103C20009F918F917F916F915F914F913F912F91D4
:103C30000F900FBE0F901F9018951F920F920FB606
:103C40000F9211242F933F934F935F936F937F9322
:103C50008F939F93AF93BF93CF93DF93EF93FF9394
:103C6000C091E900CF708091EC00D82FD17080FD19
:103C7000D0E81092E9008091F000877F8093F000F7
:103C800078940E94611E1092E9008091F000886093
:103C90008093F000CD2BCF70C093E900FF91EF919E
:103CA000DF91CF91BF91AF919F918F917F916F9154
:103CB0005F914F913F912F910F900FBE0F901F90EA
:103CC00018951F93CF93DF93CDB7DEB7AA970FB6A2
:103CD000F894DEBF0FBECDBFE7E7F2E08091F100C0
:103CE000819322E0EF37F207C9F70E94CC19809147
:103CF000E80083FF2EC18091770290917802492FCE
:103D000050E04A30510508F024C1FA01EE59FF4F46
:103D10000C94F11F803821F0823809F01AC108C0D4
:103D20008091730290917402992389F082600FC090
:103D300080917B028F70873008F00BC18093E9007F
:103D40008091EB0085FB882780F91092E900909123
:103D5000E800977F9093E8008093F1001092F100C3
:103D6000D1C0282F2D7F09F0F4C0882319F08230AC
:103D700061F0EFC080917902813009F0EAC09330A0
:103D800009F080E0809374022EC080917902811145
:103D90002AC080917B028F702FEF280F263008F009
:103DA000D8C08093E9002091EB0020FF1CC0933025
:103DB00021F48091EB00806214C09091EB0090613F
:103DC0009093EB0021E030E0A90102C0440F551FA1
:103DD0008A95E2F74093EA001092EA008091EB00A6
:103DE00088608093EB001092E9008091E800877F63
:103DF0008093E8000E947E1CACC08111AAC0109183
:103E000079021F778091E3008078812B8093E30013
:103E10008091E800877F8093E8000E947E1C80915B
:103E2000E80080FFFCCF8091E30080688093E3008E
:103E3000111102C082E001C083E08093760289C044
:103E40008058823008F085C08091790290917A0282
:103E50008C3D53E0950779F583E08A838AE2898374
:103E60004FB7F894DE01139620E03EE051E2E32FD5
:103E7000F0E050935700E49120FF03C0E295EF700B
:103E80003F5FEF708E2F90E0EA3010F0C79601C0D0
:103E9000C0968D939D932F5F243149F74FBF80913A
:103EA000E800877F8093E8006AE270E0CE01019627
:103EB0000E948A1B16C060917B0270917C02AE0149
:103EC0004F5F5F4F0E94CE1ABC01892B09F441C09D
:103ED0009091E800977F9093E80089819A810E94F1
:103EE000E81B8091E8008B778093E80032C080382F
:103EF00081F58091E800877F8093E80080917202CD
:103F00008093F1008091E8008E7772CF811121C0FB
:103F10008091790290917A0299270297D4F4809146
:103F2000E800877F8093E800809179028093720295
:103F30000E947E1C80917202811106C08091E30074
:103F400087FD02C081E001C084E0809376020E9478
:103F5000B8198091E80083FF0AC08091E800877F4C
:103F60008093E8008091EB0080628093EB00AA963A
:103F70000FB6F894DEBF0FBECDBFDF91CF911F917A
:103F800008950895CF93809176028823A1F0C0917F
:103F9000E900CF709091EC00892F817090FD80E84E
:103FA000C82B1092E9008091E80083FD0E94611EF9
:103FB000CF70C093E900CF91089597FB072E16F4B8
:103FC000009407D077FD09D00E94F71F07FC05D0A9
:103FD0003EF4909581959F4F0895709561957F4F20
:103FE0000895EE0FFF1F0590F491E02D0994AA1B90
:103FF000BB1B51E107C0AA1FBB1FA617B70710F0D4
:10400000A61BB70B881F991F5A95A9F78095909505
:10401000BC01CD010895FB01DC0104C08D9101902C
:10402000801921F441505040C8F7881B990B08951E
:10403000F999FECF92BD81BDF89A992780B5089570
:10404000A8E1B0E042E050E00C944C20262FF99912
:10405000FECF92BD81BDF89A019700B4021639F0E7
:104060001FBA20BD0FB6F894FA9AF99A0FBE0895B8
:104070000396272F0E9427200E942620252F0E948A
:104080002720242F0C9427200196272F0E942720D9
:104090000C942620DC01CB01FC01F999FECF06C06F
:1040A000F2BDE1BDF89A319600B40D9241505040F6
:0840B000B8F70895F894FFCF62
:1040B800C800F401280850011E0A1401FC181F1931
:1040C80000198F198B19FF1801E200E900EA00B501
:1040D80000B600B700CD008301CC008A019201949C
:1040E800012102230224022502260227022A02B302
:1040F80000B4006F007000818283E200E900EA00EA
:10410800B500B600B700CD008301CC008A0192014A
:1041180094012102230224022502260227022A02F0
:10412800B300B4006F00700081828394959697F075
:04413800F1F4F500A9
:00000001FF
